:1000000012C08FC1189518951895189518951895C0
:100010001895189518951895189518951895189578
:1000200018951895CDC28FED8DBFC0ECE4ED4E2E26
:10003000DD275D2EEEE7F0E0A0E6B0E088278D93A7
:100040003197E9F766248FEF87BB80E381BB8FECA4
:1000500082BB81EC80BF81E083BF8CE086BF85B727
:10006000836085BF81EF8FBD81E08EBD80E481BD5F
:10007000C198C798C598C698C09895988FEF90E09A
:1000800090934B0080934A008FEF90E0909349004B
:100090008093480080E08093630000B34BE004232A
:1000A000A1E60C93009161000B3009F014C080E0D0
:1000B00090E090934B0080934A0080E090E0909312
:1000C00049008093480084EF91E0DBD288B392E04E
:1000D000892788BBF8CF00916100003009F004C087
:1000E00080E18093660035C000916100013009F025
:1000F00004C088E0809366002CC00091610002304B
:1001000009F004C084E08093660023C00091610080
:10011000033009F004C082E0809366001AC00091A9
:100120006100083009F004C081E08093660011C0CE
:1001300000916100093009F004C082E080936600FC
:1001400008C0009161000A3009F003C081E080938B
:10015000660000B34BE00423A1E60C93009161001C
:100160000A3081E009F080E08F930091610009304E
:1001700081E009F080E09F91892B882309F432C047
:10018000809160008F77809360008AE080936A009E
:1001900080E0882EA8E00C914AE0041710F009F0E6
:1001A00020C0E4E3F6E0A8E08C919927A8E0AD90A8
:1001B000A0E7AA0D85D2EEE5F6E0A8E08C9199279C
:1001C000A8E0AD90A1E8AA0D7BD2E2E5F6E0A8E0B8
:1001D0008C919927A8E0AD90A2E9AA0D71D28394E1
:1001E000D9CF60C08091600080688093600080E11A
:1001F00080936A0000916600003109F02AC080E017
:10020000882EA8E00C9140E1041710F009F020C0FE
:10021000EEE5F6E0A8E08C919927A8E0AD90A0E784
:10022000AA0D4ED2EEE5F6E0A8E08C919927A8E061
:10023000AD90A1E8AA0D44D2EEE5F6E0A8E08C91DD
:100240009927A8E0AD90A2E9AA0D3AD28394D9CF1C
:1002500029C080E0882EA8E00C9140E1041710F03E
:1002600009F020C0E2E2F6E0A8E08C919927A8E02E
:10027000AD90A0E7AA0D24D2EEE5F6E0A8E08C91BF
:100280009927A8E0AD90A1E8AA0D1AD2E0E4F6E023
:10029000A8E08C919927A8E0AD90A2E9AA0D10D210
:1002A0008394D9CF00916A0042E015D2ABE64C931B
:1002B0000091660042E00FD2AEE64C9380E080935E
:1002C0006700809067008FEF90E090934B008093E1
:1002D0004A0080E090E09093490080934800C798DE
:1002E000C598C69AC09A809160008064809360002F
:1002F00084EF91E0C6D180E080936900ACE6E3D161
:10030000809160008F7D80936000C19A80E080932F
:100310006F0078948BB780648BBF0000FECFF89499
:10032000FFCFF894959880E080936900869914C077
:1003300080EC80936200A0E68C9186FB0EF006C0F4
:10034000082D40916600041B802E05C0082D4091A9
:100350006600040F802E13C080E480936200A0E644
:100360008C9186FB0EF006C0082D40916600040FAC
:10037000802E05C0082D40916600041B802EA8E049
:100380000C9140E0041709F03CC0949A0091680079
:10039000003280E010F009F081E08F930091680056
:1003A0000E3281E010F009F080E09F9189238823CC
:1003B00009F40BC08091600080618093600080919F
:1003C00060008F7D809360001BC000916800003347
:1003D00008F40BC08091600080628093600080917F
:1003E00060008F7E809360000BC0009168000E312A
:1003F00010F009F005C0809160008F7E809360004E
:1004000001C09498A8E00C9140E8041710F009F09E
:1004100001C016C0082D40916E00040F802EACE67E
:100420000D911C9141E050E0040F151FACE60D93B7
:100430001C930091630040916200040FA3E60C93AB
:10044000A8E00C91AAE64C91041710F009F001C045
:100450000CC0082D40916E00041B802E009163009B
:1004600040916200040FA3E60C93082D40916A00AE
:10047000040F902EA9E00C91AAE64C91041710F0FD
:1004800009F001C005C000916B00492D041B902E9E
:10049000A0E68C9185FB0EF00FC0A8E0AD90A1E81E
:1004A000AA0D8C9180936400A9E0AD90A1E8AA0DFB
:1004B0008C918093650022C0A0E68C9184FB0EF0A5
:1004C0000FC0A8E0AD90A2E9AA0D8C9180936400C2
:1004D000A9E0AD90A2E9AA0D8C91809365000EC0B1
:1004E000A8E0AD90A0E7AA0D8C9180936400A9E0EC
:1004F000AD90A0E7AA0D8C9180936500A4E68C9145
:10050000992790934B0080934A00A5E68C919927F8
:10051000909349008093480000916300003009F0F7
:1005200011C0C798C598C69A009164000F3F09F0A2
:1005300002C0C09801C0C09A80916000806480931E
:1005400060003CC000916300003409F011C0C59800
:10055000C698C09A009165000F3F09F002C0C79885
:1005600001C0C79A809160008F7B8093600026C095
:1005700000916300003809F011C0C098C698C79A6E
:10058000009164000F3F09F002C0C59801C0C59AF0
:100590008091600080648093600010C0C098C7980C
:1005A000C59A009165000F3F09F002C0C69801C0CE
:1005B000C69A809160008F7B809360007894189534
:1005C000AFE68C918F5F8C93A9E68C918F5F8C93B3
:1005D000009169000F3308F405C0959A8CEB809365
:1005E000690001C0959800916F00053008F418C0AB
:1005F00080E080936F00ACE60D911C910E3F50E0BF
:10060000150710F009F001C005C08EEF90E0ACE6D0
:100610008D939C93ACE68C91A8E68C93ACE653D07A
:100620001895FFE6CDB59D87715D4B3A2B1E130BD8
:1006300005010000FFD7B08B694B311C0C03000093
:10064000FFD6AE8A6A503C302C2C2C2C2C2C2C2C17
:100650002C00FFBE8355362C2C2C2C2C2C004B4B05
:100660004B4B4B4B4B4B4B4B4B4B4B4B4B4B4B0025
:100670003197F1F70895689462F80895E89462F864
:100680000895EF93FF93EE27E82BE92B31F0E8E88C
:10069000F3E13197F1F70197D1F7FF91EF910895C9
:1006A000C89531960020089591E005C092E003C0FE
:1006B00094E001C098E0F4DF0D929A95E1F7089577
:1006C000E80FF91FF1CF82E001C084E099279D93E4
:1006D0008A95E9F70895FF935527F8E0469508F4C1
:0E06E000500F57954795FA95D1F7FF91089561
:00000001FF
